:10800000FEDF07EA000000000000000000000000A2
:108010000000000000000000000000000000000060
:108020000000000000000000000000000000000050
:108030000000000000000000000000000000000040
:108040000000000000000000000000000000000030
:02000004001FDB
:020000040020DA
:1000000002D3A0E3A60000EBFEFFFFEA001080E5AC
:100010001EFF2FE1B010C0E11EFF2FE10010C0E570
:100020001EFF2FE1000090E51EFF2FE10E00A0E172
:100030001EFF2FE110FF2FE11EFF2FE108402DE9E9
:1000400008009FE5F6FFFFEB0840BDE81EFF2FE12B
:100050005450212008402DE91C009FE5F0FFFFEBE4
:10006000010010E3FBFFFF0A10009FE5ECFFFFEB30
:100070000840BDE8FF0000E21EFF2FE154502120A0
:100080004050212008402DE90C009FE5E4FFFFEBE4
:100090000840BDE8010000E21EFF2FE1545021207E
:1000A00010402DE90040A0E11C009FE5DCFFFFEBC4
:1000B000200010E3FBFFFF0A0410A0E10C009FE505
:1000C000D1FFFFEB1040BDE81EFF2FE1545021206F
:1000D0004050212008402DE910009FE5D0FFFFEBA4
:1000E000010C10E3FBFFFF1A0840BDE81EFF2FE1E3
:1000F0005450212038402DE90050A0E12040A0E3D9
:10010000044044E23534A0E10F3003E2090053E338
:100110003700838230008392E0FFFFEB000054E35E
:10012000F6FFFF1A2000A0E33840BDE8DBFFFFEA3E
:1001300008402DE9EEFFFFEB0D00A0E3D7FFFFEB3A
:100140000A00A0E30840BDE8D4FFFFEA10402DE913
:10015000D8009FE50110A0E3ABFFFFEBD0009FE5C7
:100160000010A0E3A8FFFFEBC8009FE50010A0E38C
:10017000A5FFFFEBC0009FE50310A0E3A2FFFFEB8C
:10018000B8009FE50010A0E39FFFFFEBA0009FE5F4
:100190000010A0E39CFFFFEBA4009FE5C610A0E3C6
:1001A00099FFFFEB9C109FE59C009FE596FFFFEBFE
:1001B00098009FE59AFFFFEB3F1AC0E3121A81E314
:1001C00088009FE590FFFFEB84009FE50010A0E30F
:1001D0008DFFFFEB0040A0E30400A0E1014084E2BA
:1001E00094FFFFEB960054E3FAFFFF1A64009FE5CB
:1001F0000319A0E384FFFFEB0040A0E30400A0E1AB
:10020000014084E28BFFFFEB960054E3FAFFFF1AF4
:1002100040009FE50010A0E37BFFFFEB14009FE58B
:100220000310A0E378FFFFEB1040BDE81EFF2FE1B5
:100230000450212044502120605021204C50212086
:1002400050502120485021200E01000068502120EC
:1002500004002020940020209800202010402DE948
:100260001C409FE5F918A0E30400A0E166FFFFEB46
:100270000400A0E10C109FE563FFFFEB1040BDE818
:100280001EFF2FE108B400200002F90008402DE90C
:1002900008009FE562FFFFEB0840BDE81EFF2FE16D
:1002A00020B40020F0472DE9A7FFFFEB08029FE5EF
:1002B0009EFFFFEB5CFFFFEB9CFFFFEB0209A0E35F
:1002C0009AFFFFEBE4FFFFEBF0719FE5F0619FE524
:1002D0001500A0E371FFFFEBEBFFFFEB0040A0E197
:1002E000020000EA66FFFFEB000050E30A00001A7C
:1002F000E5FFFFEB000064E0070050E1F8FFFF9A24
:100300001500A0E365FFFFEB5DFFFFEB3D4884E2D6
:10031000000050E3094C84E2F4FFFF0A02A9A0E3C5
:100320000080A0E3C040A0E30190A0E348FFFFEB02
:10033000C00054E30050A0E13600000A2500009AF6
:10034000C10054E35100000AC20054E34900001AFE
:10035000FF3069E2000053E15400000A1800A0E3F6
:100360004EFFFFEB1800A0E34CFFFFEB1800A0E3EB
:100370004AFFFFEB1800A0E348FFFFEB1800A0E3E3
:1003800046FFFFEBC0FFFFEB0040A0E1BEFFFFEB2D
:10039000000064E0060050E1FBFFFF9A0D00A0E3BF
:1003A0003EFFFFEB0A00A0E33CFFFFEB0A00A0E3E7
:1003B0003AFFFFEB0C019FE55CFFFFEB44FFFFEB17
:1003C000000000EA22FFFFEB2DFFFFEB000050E3EF
:1003D000FBFFFF1ABDFFFFEA800054E32500001A6F
:1003E000FF8008E2080050E1DBFFFF1A0600A0E3EF
:1003F0002AFFFFEB16FFFFEBC040A0E3019089E26C
:10040000C00054E30580A0E180A08AE2FF9009E2E9
:100410000050A0E1C8FFFF1A010050E32000000ACD
:10042000040050E3CCFFFF1A0600A0E31BFFFFEB24
:1004300095FFFFEB0050A0E193FFFFEB000065E0AC
:10044000060050E1FBFFFF9A0D00A0E313FFFFEB56
:100450000A00A0E311FFFFEB0A00A0E30FFFFFEB90
:1004600064009FE531FFFFEB19FFFFEB0209A0E3FA
:10047000EFFEFFEBACFFFFEA0450CAE7014084E265
:10048000FF0054E3058088E0A7FFFF1AB2FFFFEAF0
:10049000090050E1B0FFFF1A098088E0C240A0E3E4
:1004A000A1FFFFEA0080A0E1C140A0E39EFFFFEAB8
:1004B000038088E00040A0E39BFFFFEA78563412F7
:1004C000FF083D007F841E00ADDBBA00DADADADA1D
:040000030000800079
:00000001FF
